:10000000B6010C29A501A400B7172730A3001030B2
:1000100015200330A300E8301520A301643015201B
:10002000A3010A30152024082028A2002508A100D9
:100030002408A000D5202008031DB713B71B080013
:10004000303EA7000711871007108316071187108D
:100050000710F030860583122708B6184D283A306D
:10006000A1009830AA203330A60062201330A100EE
:100070008830AA2062206430A92062206430A92040
:100080002230A600622028304C200C304C20063054
:100090004C20B61427084D283614A600361C5B28C1
:1000A0008710033C031C602860200730A100D0307B
:1000B000AA20031408003614FE3C031907298714EC
:1000C000A60E361C36100715F030860526080F39A7
:1000D00086040711A60E361862283230A9200314B0
:1000E0000800A000A00DA00DA00D3830A0058130A3
:1000F00020049F000030A1003230AA201F151F19D4
:100100007F281E08A10083161E08072903178D00EB
:1001100083168C130C1483120C08072903178C0008
:1001200083168C130C1555308D00AA308D008C145D
:100130008C1898280C110729A301A200FF30A207F0
:10014000031CA307031C07290330A100E730AA20E2
:100150009E28A101FC3EA000A109031CB528FF3088
:100160000000A0070318B028A0076400A10FAF2863
:100170000800A2000230C528A2000330C528A20052
:100180000130C528A2000430C528A8002308210298
:10019000031DCC2822082002043003180130031963
:1001A00002302805031DFF3007291030A600A501E5
:1001B000A401210DA40DA50D2208A4022308031CEF
:1001C000230FA5020318EB282208A407230803180D
:1001D000230FA5070310A00DA10DA60BD9282008F9
:1001E00007291030A800A101A001A70CA60C031C30
:1001F000FF282208A00723080318230FA107A10C3A
:10020000A00CA50CA40CA80BF5282408072983131F
:1002100003138312640008008316DF3085008230E8
:100220009F0070308600811387018312850186014B
:1002300087018A11F929861783168613FE308312E7
:100240008A01212001308A01212048308A012120A1
:1002500069308A01212020308A01212047308A011B
:10026000212075308A01212079308A0121207330C4
:100270008A01212021308A01212020308A01212079
:1002800072308A01212065308A01212076308A016E
:10029000212031308A0121202E308A012120313065
:1002A0008A0121200330A300E8308A019D20FE301E
:1002B0008A012120C0308A01212050308A0121206A
:1002C00072308A0121206F308A01212064308A0136
:1002D000212075308A01212063308A012120653078
:1002E0008A01212064308A01212020308A012120C6
:1002F00062308A01212079308A01212020308A0150
:10030000212041308A0121204F308A0121205230A2
:100310008A01212063308A0121200330A300E830C4
:100320008A019D20080003308A017120BC00210849
:10033000BD000A308A019C20080002308A01712029
:10034000C2002108C3000A308A019C200800013045
:100350008A017120C6002108C7000A308A019C204A
:10036000080000308A017120CA002108CB000A3041
:100370008A019C200800FE308A012120C0308A01B9
:10038000212052308A01212065308A0121206D30E0
:100390008A01212061308A01212069308A012120CF
:1003A0006E308A0121205508A50054088A010320D7
:1003B00030308A01212073308A0121203A308A01AD
:1003C00021203F08A5003E088A01032063308A01EE
:1003D000212020308A01212020308A012120203054
:1003E0008A01212020308A01212020308A01212009
:1003F00008000713831607138312071283160712C8
:100400008312871183168711831285128316851232
:1004100083128A011B213E30E2003E30E3003E3071
:10042000E4003E30E50064308A019C2064008A11BB
:10043000061F132A861383168613FE3083128A0141
:10044000212001308A01212042308A0121203A30C6
:100450008A01212054308A01212069308A0121201B
:1004600072308A01212065308A01212020308A01E2
:10047000212068308A01212065308A0121206130E5
:100480008A01212074308A01212020308A01212014
:1004900063308A0121206F308A0121206E308A0169
:1004A000212074308A012120FE308A012120C030B1
:1004B0008A01212059308A0121203A308A012120E5
:1004C0004D308A0121206F308A01212074308A0149
:1004D00021206F308A01212072308A0121202030B2
:1004E0008A01212064308A01212072308A01212072
:1004F00065308A01212073308A01212073308A01FE
:1005000021200130A3002C308A019D20071383167F
:10051000071383120712831607128312871183169B
:100520008711831285128316851264008A11831243
:10053000061EA02A64008A15861E58288A01862A6B
:1005400064308A019C2064008A11061EA02A0530AE
:100550008A018620DE00DF0109308A018620D8006A
:10056000D9010A308A018620DA00DB010B308A01CA
:100570008620DC00DD01E001E101FE308A0121205E
:1005800001308A01212054308A01212065308A01FE
:1005900021206D308A01212070308A0121205F08DE
:1005A000A5005E088A0103203A308A0121205908FB
:1005B000A50058088A0103203A308A0121205B08EF
:1005C000A5005A088A0103203A308A0121205D08DB
:1005D000A5005C088A010320FE308A012120C0307A
:1005E0008A01212043308A01212068308A0121209C
:1005F00061308A0121206E308A01212067308A0112
:10060000212065308A0121203F308A0121202030BD
:100610008A01212052308A0121203A308A0121208A
:100620004E308A01212020308A01212042308A0167
:1006300021203A308A01212059308A012120C830F6
:100640008A019C2064008A11061E2C2B64008A11EA
:10065000061FBE2D8A01222B64308A019C20640073
:100660008A11061E2C2BFE308A01212001308A01BE
:10067000212041308A01212020308A01212054305C
:100680008A01212065308A0121206D308A012120D4
:1006900070308A0121202E308A01212020308A01E9
:1006A000212073308A01212065308A012120743095
:1006B0008A0121203D308A0121205F08A5005E08C3
:1006C0008A010320FE308A012120C0308A012120C6
:1006D00052308A0121203A308A0121204E308A018D
:1006E000212065308A01212078308A012120743050
:1006F0008A01212020308A01212059308A012120BD
:100700003A308A01212044308A0121206E308A014A
:10071000212020308A01212042308A0121203A30D4
:100720008A01212055308A01212070308A01212040
:10073000C8308A019C2064008A11061EA92B64001F
:100740008A11861EBC2B64008A11061FD22B8A01D7
:100750009B2BDE0A0319DF0A5E08A0005F08A100D8
:10076000A30150308A01C2208A11031DBA2B5030D8
:10077000DE00DF018A01332B0130DE020030031C72
:10078000013EDF025E08A0005F08A100A3010A305D
:100790008A01BF208A11031DD02B0A30DE00DF0141
:1007A0008A01332B32308A019C2064008A11061F93
:1007B000D22BFE308A01212001308A0121204230D3
:1007C0008A01212020308A01212054308A012120F1
:1007D00065308A0121206D308A01212070308A0124
:1007E00021202E308A01212020308A0121207330DF
:1007F0008A01212065308A01212074308A0121205C
:100800003D308A0121205908A50058088A0103209B
:10081000FE308A012120C0308A01212052308A0115
:1008200021203A308A0121204E308A012120653072
:100830008A01212078308A01212074308A01212008
:1008400020308A01212059308A0121203A308A0142
:10085000212044308A0121206E308A01212020305D
:100860008A01212042308A0121203A308A01212048
:1008700055308A01212070308A012120C8308A0138
:100880009C2064008A11061E4F2C64008A11861E6B
:10089000622C64008A11061F782C8A01412CD80A28
:1008A0000319D90A5808A0005908A100A301503023
:1008B0008A01C2208A11031D602C5030D800D90152
:1008C0008A01D92B0130D8020030031C013ED90225
:1008D0005808A0005908A100A3010A308A01BF20CE
:1008E0008A11031D762C0A30D800D9018A01D92B30
:1008F00032308A019C2064008A11061F782CFE3059
:100900008A01212001308A01212043308A012120DF
:1009100020308A01212054308A01212065308A014B
:1009200021206D308A01212070308A0121202E3053
:100930008A01212020308A01212073308A01212060
:1009400065308A01212074308A0121203D308A01DE
:1009500021205B08A5005A088A010320FE308A0185
:100960002120C0308A01212052308A0121203A30D2
:100970008A0121204E308A01212065308A01212000
:1009800078308A01212074308A01212020308A01A8
:10099000212059308A0121203A308A012120443017
:1009A0008A0121206E308A01212020308A012120F5
:1009B00042308A0121203A308A01212055308A01B3
:1009C000212070308A012120C8308A019C206400D7
:1009D0008A11061EF52C64008A11861E082D6400FB
:1009E0008A11061F1E2D8A01E72CDA0A0319DB0A79
:1009F0005A08A0005B08A100A30150308A01C22060
:100A00008A11031D062D5030DA00DB018A017F2C8C
:100A10000130DA020030031C013EDB025A08A0005C
:100A20005B08A100A3010A308A01BF208A11031DBF
:100A30001C2D0A30DA00DB018A017F2C32308A015A
:100A40009C2064008A11061F1E2DFE308A01212081
:100A500001308A01212044308A01212020308A017E
:100A6000212054308A01212065308A0121206D30F7
:100A70008A01212070308A0121202E308A01212014
:100A800020308A01212073308A01212065308A01BB
:100A9000212074308A0121203D308A0121205D0807
:100AA000A5005C088A010320FE308A012120C030A5
:100AB0008A01212052308A0121203A308A012120E6
:100AC00047308A0121206F308A01212020308A019D
:100AD000212059308A0121203A308A0121204430D6
:100AE0008A0121206E308A01212020308A012120B4
:100AF00042308A0121203A308A01212055308A0172
:100B0000212070308A012120C8308A019C20640095
:100B10008A11061E952D64008A11861EA82D640078
:100B20008A11061FBE2D8A01872DDC0A0319DD0AF2
:100B30005C08A0005D08A100A30150308A01C2201A
:100B40008A11031DA62D5030DC00DD018A01252D00
:100B50000130DC020030031C013EDD025C08A00015
:100B60005D08A100A3010A308A01BF208A11031D7C
:100B7000BC2D0A30DC00DD018A01252D64308A019C
:100B80009C2064008A11061FBE2D031705308D00BE
:100B900003135E088A018E20031709308D000313AA
:100BA00058088A018E2003170A308D0003135A0853
:100BB0008A018E2003170B308D0003135C088A0115
:100BC0008E2007138316071383120712831607124A
:100BD000831287118316871183128512831685125B
:100BE0008312E00A0319E10A6008A0006108A1006D
:100BF0000E30A30010308A01BF208A11031DDB2FA5
:100C00008A0193213C08A6003D08A7007D30A20080
:100C1000A3018A01F120B2002508B3003208A00028
:100C20003308A100A2010130A3008A01D520BE0033
:100C30002108BF008A019D214208A6004308A700A1
:100C40007D30A200A3018A01F120B2002508B30083
:100C50003208A0003308A100A2010130A3008A01DC
:100C6000D520C4002108C5008A01A7214608A60096
:100C70004708A7007D30A200A3018A01F120B2003D
:100C80002508B3003208A0003308A100A2010130FA
:100C9000A3008A01D520C8002108C9008A01B1211A
:100CA0004A08A6004B08A7007D30A200A3018A01D4
:100CB000F120B2002508B3003208A0003308A100DB
:100CC000A2010130A3008A01D520CC002108CD006B
:100CD000FE308A01212001308A01212041308A0121
:100CE00021205F08A5005E088A0103203A308A01AE
:100CF000212042308A0121205908A50058088A0184
:100D000003203A308A01212043308A0121205B08E8
:100D1000A5005A088A0103203A308A012120443074
:100D20008A0121205D08A5005C088A01032020308B
:100D30008A01212020308A012120FE308A012120D1
:100D4000C0308A01212062088A0121203F08A500C5
:100D50003E088A01032020308A012120FE308A01CA
:100D60002120C0308A012120FE308A012120143048
:100D70008A012120FE308A01212014308A0121209D
:100D8000FE308A01212014308A0121203A308A0164
:100D9000212063088A0121204508A50044088A0112
:100DA000032020308A012120FE308A012120C0301A
:100DB0008A012120FE308A01212014308A0121205D
:100DC000FE308A01212014308A012120FE308A0160
:100DD000212014308A012120FE308A012120143084
:100DE0008A012120FE308A01212014308A0121202D
:100DF000FE308A01212014308A012120FE308A0130
:100E0000212014308A0121203A308A0121206408EF
:100E10008A0121204908A50048088A0103202030C2
:100E20008A012120FE308A012120C0308A01212040
:100E3000FE308A01212014308A012120FE308A01EF
:100E4000212014308A012120FE308A012120143013
:100E50008A012120FE308A01212014308A012120BC
:100E6000FE308A01212014308A012120FE308A01BF
:100E7000212014308A012120FE308A0121201430E3
:100E80008A012120FE308A01212014308A0121208C
:100E9000FE308A01212014308A012120FE308A018F
:100EA000212014308A012120FE308A0121201430B3
:100EB0008A0121203A308A01212065088A012120F7
:100EC0004D08A5004C088A01032020308A0121200A
:100ED00064008A11061FF9293E08A0003F08A100FE
:100EE0005F08A3005E088A01C2208A11031D802FBB
:100EF00007138316071383122D30E2008A11862F01
:100F000007178316071383122B30E2004408A00052
:100F10004508A1005908A30058088A01C2208A1177
:100F2000031D9A2F07128316071283122D30E30038
:100F30008A11A02F07168316071283122B30E300A5
:100F40004808A0004908A1005B08A3005A088A01CC
:100F5000C2208A11031DB42F8711831687118312B3
:100F60002D30E4008A11BA2F87158316871183125A
:100F70002B30E4004C08A0004D08A1005D08A30040
:100F80005C088A01C2208A11031DCE2F85128316A8
:100F9000851283122D30E5008A11D42F8516831611
:100FA000851283122B30E5000330A300CA308A017A
:100FB0009D208A01F12D0713831607138312071250
:100FC00083160712831287118316871183128512E5
:100FD00083168512FE3083128A01212001308A0196
:100FE00021204F308A01212076308A01212065306E
:100FF0008A01212072308A01212020308A0121209B
:1010000031308A01212020308A01212068308A0174
:1010100021206F308A01212075308A012120723011
:101020008A01212020308A01212021308A012120BB
:10103000FE308A012120C0308A01212048308A01F7
:10104000212065308A01212061308A0121207430FD
:101050008A01212020308A0121206F308A0121203D
:1010600066308A01212066308A01212020308A01E1
:10107000212062308A01212079308A01212020300C
:101080008A01212074308A01212069308A012120BF
:101090006D308A01212065308A0121208613831654
:1010A0008613831264008A11061FF9298A155228B3
:1010B00064308A019C2064008A15861E5828861395
:1010C00083168613063083128A018620E8000730D3
:1010D0008A018620E70008308A018620C000C1010D
:1010E00009308A018620E6006708A600A701A20150
:1010F0000130A3008A01F120B2002508B30068087E
:101100003207D40033080318013ED500FE308A01AF
:10111000212001308A01212053308A01212074309E
:101120008A0121206F308A01212070308A0121201C
:1011300020308A01212074308A01212065308A0103
:1011400021206D308A01212070308A0121202E302B
:101150008A0121203D308A0121204108A500400854
:101160008A010320FE308A012120C0308A0121201B
:1011700052308A0121203A308A0121204E308A01E2
:10118000212065308A01212078308A0121207430A5
:101190008A01212020308A01212059308A01212012
:1011A0003A308A01212044308A0121206E308A01A0
:1011B000212020308A01212042308A0121203A302A
:1011C0008A01212055308A01212070308A01212096
:1011D00096308A019C2064008A15061EF928640056
:1011E0008A15861E0C2964008A15061F22298A1575
:1011F000EB28C00A0319C10A4008A0004108A10059
:10120000A3015A308A01C2208A15031D0A295A30C7
:10121000C000C1018A1586280130C0020030031CBD
:10122000013EC1024008A0004108A100A3010A300C
:101230008A01BF208A15031D20290A30C000C10180
:101240008A15862864308A019C2064008A15061F4E
:101250002229FE308A01212001308A0121205430C8
:101260008A01212069308A0121206D308A012120E4
:1012700065308A01212072308A0121203D308A01A7
:1012800021205508A50054088A01032030308A0126
:10129000212073308A01212065308A0121206330AA
:1012A0008A012120FE308A012120C0308A012120BC
:1012B00052308A0121203A308A0121204E308A01A1
:1012C000212065308A01212078308A012120743064
:1012D0008A01212020308A01212059308A012120D1
:1012E0003A308A01212044308A0121206E308A015F
:1012F000212020308A01212042308A0121203A30E9
:101300008A01212055308A01212070308A01212054
:1013100096308A019C2064008A15061E9929640073
:101320008A15861EAE2964008A15061FC4298A15EF
:101330008B29D40A0319D50A5408A0005508A10026
:10134000FD30A30020308A01C2208A15031DAC297C
:101350002030D400FD30D5008A1529290130D4026F
:101360000030031C013ED5025408A0005508A1001E
:10137000A30101308A01BF208A15031DC229013053
:10138000D400D5018A15292964308A019C20640083
:101390008A15061FC429FE308A01212001308A01E6
:1013A00021204C308A0121206F308A0121207730A2
:1013B0008A01212065308A01212072308A01212092
:1013C00044308A01212075308A01212074308A013D
:1013D000212079308A0121203D308A0121206608B0
:1013E0008A01022025308A012120FE308A01212035
:1013F000C0308A01212052308A0121203A308A01EE
:1014000021204E308A01212078308A01212020308D
:101410008A01212059308A0121203A308A01212075
:1014200044308A0121206E308A01212020308A0137
:10143000212042308A0121203A308A012120553072
:101440008A01212070308A01212096308A019C2057
:1014500064008A15061E362A64008A15861E412AF3
:1014600064008A15061F4C2A8A15282AE60A640099
:10147000463066028A15031C3F2A4630E6008A156C
:10148000CB29E6036400033066028A1503184A2A52
:101490000230E6008A15CB295408E8005408A00061
:1014A0005508A100A2010130A3008A01D520E70060
:1014B000031706308D00031368088A018E20031776
:1014C00007308D00031367088A018E200317083048
:1014D0008D00031340088A018E20031709308D0008
:1014E000031366088A018E20FE308A012120013014
:1014F0008A01212043308A01212079308A0121206C
:1015000063308A0121206C308A01212069308A01F0
:10151000212063308A01212061308A0121206C3032
:101520008A01212020308A01212064308A01212073
:1015300072308A01212065308A01212073308A01AE
:10154000212073308A01212020308A0121203F3060
:101550008A012120FE308A012120C0308A01212009
:1015600059308A0121203A308A0121204E308A01E7
:1015700021206F308A01212020308A012120423031
:101580008A0121203A308A01212059308A01212004
:1015900065308A01212073308A01212064008A1578
:1015A000861ED82A64008A15061E882B8A15CE2A24
:1015B000FE308A01212001308A01212044308A0135
:1015C000212075308A01212074308A012120793050
:1015D0008A0121203D308A01212066088A010220EB
:1015E00025308A0121203A308A01212043308A01A6
:1015F000212075308A01212074308A0121203D305C
:101600008A0121204108A50040088A010320633097
:101610008A0121208A01BB21861783168613831233
:10162000D201D3015208A0005308A100B630A30094
:101630006C308A01BF208A15031D452B07178316BE
:10164000071303108312660DB200B301B30D330804
:10165000A10032088A01AA200713831607138312F8
:101660006608643CB2000030031CFF3EB300031068
:10167000B20DB30D3308A10032088A01AA20D20AA4
:101680000319D30A8A15031D122B03308A01712016
:10169000BC002108BD003C08A6003D08A7007D3025
:1016A000A200A3018A01F120B2002508B30032088C
:1016B000A0003308A100A2010130A3008A01D520B7
:1016C000BE002108BF000130D4020030031C013EDF
:1016D000D5028A01BB2164008A11061FF92954082A
:1016E000A0005508A100A30100308A01B9208A1585
:1016F000031DBF2C3E08A0003F08A1004108A30025
:1017000040088A01BC208A15031DE72C8A15102B7E
:10171000FE308A01212001308A01212066088A01D9
:10172000022025308A01212074308A0121206F3067
:101730008A0121200A306607B200B301B30D3308D5
:10174000A50032088A01032025308A0121203A3081
:101750008A01212043308A01212075308A0121200D
:1017600074308A0121203D308A0121204108A500E2
:1017700040088A01032063308A0121208A01BB21AD
:101780008617831686138312D001D1015008A0005A
:101790005108A100A30114308A01BF208A15031D3E
:1017A0001D2CD201D3015208A0005308A10004301F
:1017B000A3007D308A01BF208A15031D172C07174F
:1017C0008316071303108312660DB200B301B30D25
:1017D0005008B20751080318013EB3073308A100AF
:1017E00032088A01AA2007138316071383125008B0
:1017F000C83CB2005108031C013E003CB30003107A
:10180000660DB400B501B50D34083202B4003508D8
:10181000031C013E3302B5003508A10034088A01DB
:10182000AA20D20A0319D30A8A15031DD32BD00A82
:101830000319D10A8A15031DC62B86138316861336
:1018400083121330D000D1015008A0005108A1002C
:10185000A30101308A01C2208A15031D7C2CD2010C
:10186000D3015208A0005308A1000430A3007C302B
:101870008A01BF208A15031D752C071783160713CD
:1018800003108312660DB200B301B30D5008B20706
:1018900051080318013EB3073308A10032088A013A
:1018A000AA2007138316071383125008C83CB200FE
:1018B0005108031C013E003CB3000310660DB40048
:1018C000B501B50D34083202B4003508031C013EE1
:1018D0003302B5003508A10034088A01AA20D20AD3
:1018E0000319D30A8A15031D312C0130D002031CC1
:1018F000D1028A150318242C03308A017120BC0000
:101900002108BD003C08A6003D08A7007D30A200CC
:10191000A3018A01F120B2002508B3003208A0001B
:101920003308A100A2010130A3008A01D520BE0026
:101930002108BF000130D4020030031C013ED50253
:101940008A01BB2164008A11061FF9295408A000EE
:101950005508A100A30100308A01B9208A15031D92
:10196000BF2C3E08A0003F08A1004108A30040088A
:101970008A01BC208A15031DE72C8A15C02B07138A
:10198000831607138312861383168613FE30831281
:101990008A01212001308A01212046308A0121203C
:1019A00069308A0121206E308A01212069308A0144
:1019B000212073308A01212068308A0121202030C3
:1019C0008A01212021308A0121208A15522886137C
:1019D00083168613FE3083128A01212001308A018A
:1019E00021204F308A01212076308A012120653064
:1019F0008A01212072308A01212020308A01212091
:101A000074308A01212065308A0121206D308A01DD
:101A1000212070308A0121202E308A01212021309E
:0E1A20008A0121208A15522863008A15142D90
:02400E00723D01
:0E420A001E001200000032001E001E001E00EA
:00000001FF
